:10000000F128FF3FFF3FFF3FFF00030E8301BC00CD
:100010000408BB000A08BD008A017008C000850101
:100020008701860120088316850083122108831624
:1000300087008312220886002F08233F84000008CF
:10004000A200301C2628F030A20528280F30A20577
:1000500005302F0203185228FF30A1002F08003A64
:10006000031D35283D30A00086282F08013A031DC6
:100070003C283B30A00086282F08023A031D432865
:100080003730A00086282F08033A031D4A282F3056
:10009000A00086282F08043A031D51281F30A00015
:1000A000862886283F30A0002F08053A031D5B28CC
:1000B000FE30A10086282F08063A031D6228FD3075
:1000C000A10086282F08073A031D6928FB30A100EC
:1000D00086282F08083A031D7028F730A1008628CB
:1000E0002F08093A031D7728EF30A10086282F0832
:1000F0000A3A031D7E28DF30A10086282F080B3A1C
:10010000031D86283E30A000FF30A100AF0A0C304E
:100110002F02031C8D28AF01B00A0B114008F0001C
:100120003D088A003B0884003C0E8300FF0E7F0ED2
:100130000900031383123F08003A031DA228BB30B5
:10014000BF00E3283F08013A031DA9288230BF0001
:10015000E3283F08023A031DB0283E30BF00E328E1
:100160003F08033A031DB728AE30BF00E3283F081D
:10017000043A031DBE288730BF00E3283F08053A34
:10018000031DC528AD30BF00E3283F08063A031D14
:10019000CC289D30BF00E3283F08073A031DD32831
:1001A000A230BF00E3283F08083A031DDA28BF3019
:1001B000BF00E3283F08093A031DE128A730BF002C
:1001C000E3282030BF003E080B3C0318E9280B3021
:1001D000BE003E08233FF000700884003F08800006
:1001E0000800031383129F01073083169F008312B8
:1001F00085013F30831685008312860183168601B0
:1002000083128701FF30831687008B0189308100BC
:1002100001308312900007309200AF010130B1002D
:100220000230B200B301B401B501B601B701B801A3
:10023000A3010130BE000130BF0099200230BE0092
:100240003208BF0099200430A6000430BE003308F5
:10025000BF0099200530BE003408BF00992004304B
:10026000A9000730BE003508BF0099200830BE0045
:100270003608BF0099200430AC000A30BE003708B1
:10028000BF0099200B30BE003808BF009920A03075
:100290008B00071B7029B20A0A303202031C522954
:1002A000B201B10A3108023A031D5C293208043A4E
:1002B000031D5C29B101B2010130BE003108BF004D
:1002C00099200230BE003208BF009920071F66291E
:1002D0008F01C8300F0203187029071F662969298A
:1002E000871BAA29B40A0A303402031C7E29B401F0
:1002F000B30A06303302031C7E29B301B501B601EF
:10030000B701B8010430BE003308BF0099200530A2
:10031000BE003408BF0099200730BE003508BF007A
:1003200099200830BE003608BF0099200A30BE0070
:100330003708BF0099200B30BE003808BF00992055
:10034000871FA0298F01C8300F020318AA29871F11
:10035000A029A3298C1C2A2A8C1000303907F1000F
:100360003A080318013F043FF2007108B90072080F
:10037000BA0027307202031DBF2910307102031C1E
:100380002A2A1030B902031CBA032730BA02B80A6D
:100390000A303802031CE029B801B70A0A303702D4
:1003A000031CE029B701B60A0A303602031CE02913
:1003B000B601B50A06303502031CE029B501B40ABE
:1003C0000A303402031CFC29B401B30A063033029C
:1003D000031CFC29B301B20A0A303202031CF229C1
:1003E000B201B10A3108023A031DFC293208043A6D
:1003F000031DFC29B201B1010130BE003108BF006C
:1004000099200230BE003208BF0099200430A600B7
:100410000430BE003308BF0099200530BE00340808
:10042000BF0099200430A9000730BE003508BF0086
:1004300099200830BE003608BF0099200430AC0077
:100440000A30BE003708BF0099200B30BE003808C4
:10045000BF00992049292B2AFF3FFF3FFF3FFF3F65
:02400E00723FFF
:00000001FF
